:100000000C94CE020C94D0290C9406030C94060395
:100010000C9406030C9406030C9406030C9406033C
:100020000C9406030C9406030C945E200C949A1F07
:100030000C94361A0C9406030C9406030C940603D5
:100040000C9406030C9406030C9406030C9406030C
:100050000C9406030C94E9190C9406030C94060303
:100060000C9406030C9406030C9406030C940603EC
:100070000C9406030C9406030C9406030C940603DC
:100080000C9406030C9406030C9406030C940603CC
:100090000C9406030C9406030C9406030C940603BC
:1000A0000C9406030C9406030C9406031007100727
:1000B00042074207B4075C095C095C09D007AE0837
:1000C000BF08BF08B31DDA1D721FDA1D721F221E82
:1000D000451E721F341F471F00047F3F1F643214E8
:1000E000643214783C1E1E140A0522232526282972
:1000F0002A2C2D2F3032333536383A3B3D3E4042A4
:10010000434547494A4C4E5051535557595A5C5EE6
:100110006062646668696B6D6F71737577797B7DFA
:100120007F81838587898A8C8E90929496989A9CF9
:100130009E9FA1A3A5A7A8AAACAEAFB1B3B4B6B811
:10014000B9BBBCBEBFC1C2C3C5C6C7C9CACBCCCD73
:10015000CED0D1D2D2D3D4D5D6D7D7D8D9D9DADA4E
:10016000DBDBDBDCDCDCDCDCDDDDDDDDDCDCDCDCCE
:10017000DCDBDBDBDADAD9D9D8D7D7D6D5D4D3D202
:10018000D2D1D0CECDCCCBCAC9C7C6C5C3C2C1BFE0
:10019000BEBCBBB9B8B6B4B3B1AFAEACAAA8A7A544
:1001A000A3A19F9E9C9A98969492908E8C8A898700
:1001B0008583817F7D7B79777573716F6D6B6968DE
:1001C000666462605E5C5A5957555351504E4C4AB2
:1001D0004947454342403E3D3B3A3836353332305D
:1001E0002F2D2C2A29282625232205010980A1014B
:1001F000850319012AB700150126B700950175106E
:100200008100C0050C0901A101850419012AA00281
:10021000150126A002950175108100C0050109068F
:10022000A101050719E029E71500250195087501C9
:1002300081029501750881010507190029FF150044
:1002400026FF009506750881000508190129059506
:100250000575019102950175039101C009023B00EA
:10026000020100A0FA0904000001030101000921B4
:100270001101000122400007058103080001090463
:1002800001000103000000092111010001223200D8
:10029000070582032000011201000200000008107F
:1002A000CB67220002010200011803530069006EAF
:1002B00000630020005200650076002E002000320E
:1002C0000000000E034B0065006500620069006FCE
:1002D000000000040309043A003B0035001E001F23
:1002E0000020002100220023003C003D002B0014D0
:1002F000001A0008001500170000003E003F0039FA
:100300000004001600070009000A00000040004138
:1003100000E10000001D001B00060019000500425E
:10032000004300E000E200E300015100002C000067
:1003300000A800000029003A003B003C003D003EC0
:10034000003F0024002500260027002D002E004C31
:10035000002A004A001C0018000C00120013002F95
:1003600000300031004D000B000D000E000F003377
:10037000003400000028004B001100100036003748
:100380000038000000E50052004E0001512C00E64C
:1003900000E400E7000000500051004F0000004062
:1003A00000410042004300440045004C004900C6A3
:1003B0005CC75C165C3A003B003C003D003E003FE1
:1003C00000C85CC95CC35CC45C0100520001000150
:1003D000000000CA5CCB5C01000100500051004FDE
:1003E0000001000000010001000100000001000107
:1003F00000010001000100010001000100010001F5
:1004000000010000000100000001000000010001E7
:100410000001000100010001000100400041004214
:1004200000430044004500010001000100010001FB
:1004300000010001000100010001000100010001B4
:1004400000010001000100010001000000010001A5
:100450000001000100010001000100000001000195
:100460000001000100010001000100010000000185
:100470000001000100000001000100010001000175
:100480000001000100010000010101010101010161
:100490000102020202020202020203030303030337
:1004A0000303040404040404040505050505060605
:1004B00006060607070707070808080809090909C3
:1004C0000A0A0A0B0B0B0C0C0C0D0D0D0E0E0E0F69
:1004D0000F0F1010111111121213131414151516F9
:1004E000161717181819191A1A1B1B1C1D1D1E1E6A
:1004F0001F202021222223242425262627282929BB
:100500002A2B2C2D2D2E2F303132323334353637E5
:1005100038393A3B3C3D3E3F4041424344454647E3
:1005200048494A4C4D4E4F50515354555658595ABC
:100530005B5D5E5F616264656668696B6C6D6F7060
:1005400072737577787A7B7D7E8082838587888ACF
:100550008C8E8F91939596989A9C9EA0A2A3A5A706
:10056000A9ABADAFB1B3B5B7BABCBEC0C2C4C6C902
:10057000CBCDCFD1D4D6D8DBDDDFE2E4E7E9EBEEBB
:10058000F0F3F5F8FAFDFFFFAA7F55400102030CD6
:100590000D0E0F00070605040B0A090811241FBEE3
:1005A000CFEFDAE0DEBFCDBF04B603FE18C0809106
:1005B0008D0390918E03A0918F03B09190038730AB
:1005C000904BA740B04B59F410928D0310928E03BC
:1005D00010928F0310929003E0E0F8E3099511E088
:1005E000A0E0B1E0EEEDF7E502C005900D92A23E6D
:1005F000B107D9F723E0A2EEB1E001C01D92AD38FA
:10060000B207E1F70E945B0B0C94ED2B0C940000F9
:100610001F93CF93DF93CDB7DEB767970FB6F894EC
:10062000DEBF0FBECDBF4B8B5C8B6D8B7E8B8F8BFC
:10063000611110928B0386E09E01235F3F4FD90129
:10064000E82F1D92EA95E9F795E0FE017396D9012E
:1006500001900D929A95E1F79C894E895F897B897B
:100660007D879E876F87598B488BF901DE0117962E
:1006700001900D928A95E1F7CE0107960E948F2294
:1006800081113EC086E0FE013796DE011196019091
:100690000D928A95E1F7FF81E8856A857B85611572
:1006A000710531F0EF3F31F481E0FF3F19F403C0F1
:1006B00081E001C080E080FD23C02091500330E044
:1006C000C9010196877099274091810350E08417F2
:1006D000950779F1F983EA837D836C8396E0929F95
:1006E000D001939FB00D1124AF5ABC4FFE0131963B
:1006F00001900D929A95E1F7809350030E94842116
:1007000016E080918103909150038917F9F0189FAA
:10071000C00111248F5A9C4F0E948F228823B1F070
:100720008091810390E001968770992780938103DF
:10073000E8CF0E941B251092500310928103EAE437
:10074000F3E086E0DF011D928A95E9F767960FB620
:10075000F894DEBF0FBECDBFDF91CF911F910895FA
:1007600090914701992329F081FD02C02E9A0895A6
:100770002E980895811106C0662311F08EE409C0F9
:100780008BE407C0813039F4662311F089EA01C097
:100790008AEA0E94372580E008958F929F92AF9257
:1007A000BF92CF92DF92EF92FF920F931F93CF935E
:1007B000DF93CDB7DEB72A970FB6F894DEBF0FBE32
:1007C000CDBFFC010081D18083819481892B39F0D8
:1007D0001FEFD11206C091E00F3F19F403C091E062
:1007E00001C090E090FD9AC67F0185E0DE0116967B
:1007F00001900D928A95E1F7F70122818E819F8108
:10080000222349F00E94FA21182F682F8E819F81A0
:100810000E945C2403C00E943024182F2CE6129FF3
:10082000F001112439E0D39EE00DF11D1124E00FF9
:10083000F11DEE0FFF1FE952FD4F05911491F701D5
:100840008281882309F482C00E3BFCE51F07E1F09A
:1008500058F40C3B3CE5130799F00D3B9CE5190758
:1008600009F074C080E00DC0003CECE51E0709F4FF
:100870005AC008F43FC0013C2CE51207A9F066C03D
:1008800083E00E94041C6EC58091D302982F969538
:100890009695969549F1915E990F990F990F8770EA
:1008A000892B8093D30214C09091D302892F86950F
:1008B000869586958F5F8F719770843008F043C05E
:1008C000880F880F880F892B8093D3028091D302E1
:1008D000887F91E009F490E08091D30290FB80F949
:1008E0008093D3020E94FF1B8091D3028695869548
:1008F000869523C02091D302822F86958695869572
:10090000482F50E04330510554F48F5F982F990FD2
:10091000990F990F822F8770892B8093D302809132
:10092000D3028160DDCF8091D30280FF09C08E7F2A
:100930008093D3020E94FF1B80E00E944C1B12C5D3
:100940000E94211C0FC59093D302C0CF043F2CE519
:10095000120749F406E221EE40EE64EF7CE5C701A0
:100960000E94C21AFFC4053F3CE5130708F066C1A8
:10097000093D9CE5190731F407E225EE45EE69EDE6
:100980007CE5EDCF0A3DECE51E0731F408E221E0FD
:1009900045EE6AED7CE5E3CF083DFCE51F0731F449
:1009A00006E221EE41EE68ED7CE5D9CF882309F41B
:1009B0007AC11092D60204303DE5130758F40B3F7C
:1009C0008CE5180780F4C80182509C45449708F0D4
:1009D00054C109C002369DE5190729F0063AEDE534
:1009E0001E0709F04AC10E944D1390933102809373
:1009F00030020131FCE51F0709F4C6C008F042C00F
:100A000009303CE5130709F49BC000F505309CE56F
:100A1000190709F485C078F40330FCE51F0709F4D1
:100A200078C008F07AC002301C4509F0F7C0809108
:100A300030028160F1C007308CE5180709F478C0F6
:100A400008F07AC0809130028061E6C00D30ECE59C
:100A50001E0709F487C058F40B302CE5120709F47F
:100A600079C008F07BC08091300288606FC00F3081
:100A70008CE5180709F480C008F082C0809130022C
:100A8000877FCAC00E3FECE51E0709F471C000F570
:100A900005312CE5120709F485C068F403318CE5B3
:100AA000180709F475C008F095C00E941B258091B5
:100AB00030028F77B1C00C3FECE51E07A9F108F0BA
:100AC00054C00B3F1C4509F0A9C08091310240C0C1
:100AD00002303DE5130709F489C058F401159DE57E
:100AE000190709F45AC008F069C080913102826088
:100AF0002FC00236FDE51F0709F47EC0063A2DE53A
:100B0000120709F483C003301D4509F087C060E077
:100B10006EC08091300282607FC08091300216C02A
:100B200080913002886078C08091310282604FC02D
:100B300080913002806270C08091300280646CC00D
:100B40000E941B2580913002806866C0846064C06A
:100B500081603DC0809130028E7F5EC08091300206
:100B60008D7F5AC08091300216C08091310218C02A
:100B7000809131028D7F2BC0809130028F7E4CC0DE
:100B8000809130028F7D48C0809130028F7B44C0BD
:100B900080913002877F8B7F3FC0809131028D7FB3
:100BA0008E7F15C08091300282FB222720F991E0D0
:100BB000922790FB82F990FB83F92EC0809131023D
:100BC000982F909591708E7F892B90FB81F980935F
:100BD000310224C00E941B258091300287FB22270E
:100BE00020F991E0922790FB87F916C061E08EE032
:100BF00090E00E94052B12C08091300284FB2227D6
:100C000020F991E0922790FB84F906C08091300290
:100C1000982F909590FB80F980933002609130027C
:100C20001091310284E090E00E94052B612F82E256
:100C300090E00E94052B0E941B2594C3063F2CE5E3
:100C4000120731F406E221EE42EE66EF7CE587CE34
:100C5000063F3CE5130730F407E225EE44EE65EF6E
:100C60007CE57DCE073F9CE5190709F09FCE07E2A2
:100C700025EE46EE67EF7CE572CE0631ECE51E0709
:100C800021F580918C038A7A91E009F490E09093A9
:100C9000E401882311F065E301C069E28CEF92E082
:100CA0000E946C1A0FC00631FCE51F0709F040C016
:100CB0008091E401882309F478C365E38CEF92E026
:100CC0000E945F1A0E943C214DC30B35FDE51F07B2
:100CD00049F158F401153CE51307B1F00F3D1C45EF
:100CE00009F042C00E945E133DC30C359DE5190713
:100CF000D9F00D351D45C1F58091310282FB882761
:100D000080F991E0892711C00E941B25FFEF04E3C1
:100D10001CE0F15000401040E1F700C000000E94CC
:100D2000C51920C381E001C080E00E94D3241CC00B
:100D300080918C0382720D3C9CE5190709F4CEC3A7
:100D400008F0F9C2073CFCE51F0709F4B3C308F03B
:100D50003CC3043C3CE5130709F4A2C308F027C3D5
:100D6000033C1C4509F472C3F70182810081D180E4
:100D7000882359F0802F9D2D0E94FA21182F682F6B
:100D8000802F9D2D0E945C2405C0802F9D2D0E94E8
:100D90003024182F2CE6129FF001112439E0D39E45
:100DA000E00DF11D1124E00FF11DEE0FFF1FE952C0
:100DB000FD4F859194910E946C118C01982EF70142
:100DC000D280A580A2943FE0A32280918203877005
:100DD000B9F0DD20A9F0812F807F803421F080E2FE
:100DE000800F883068F08091310282FD09C082E076
:100DF0000E94B624809182038770CC24C394811111
:100E0000C12CB12EB2949FE0B9228B2D90E08C3092
:100E1000910508F051C2FC01EA5AFF4F0C94932B44
:100E2000812F807F1F70882311F01295107FDD20A5
:100E3000B9F0112309F42DC280E2800F883010F040
:100E4000911006C080918C03182B10938C0305C061
:100E500080918B03182B10938B030E943C2119C2A5
:100E6000802F0E943C28112309F426C2005E08301E
:100E700078F1992069F1109580918B0318231093D4
:100E80008B0329C0812F807F1F70803211F0129553
:100E9000107F992021F0F1E09F16D9F149C080918F
:100EA000310282FF1BC0DD2069F0112339F08091EF
:100EB0008C03182B10938C030E943C2180E00E942D
:100EC0009328FAC180E00E943C28112309F4F4C160
:100ED000812F0E9435210E943C21EEC1DD2081F04E
:100EE00080916E02AA2051F001E0A01207C0182BD9
:100EF000181709F4E1C110936E02DEC1812B10C0F6
:100F0000AA2021F021E0A21609F4D6C10E94CE1336
:100F100027C0DD2041F035E03A1508F4CDC1812F1E
:100F20000E942D25C9C184E08A1508F4C5C118C0E6
:100F3000DD2049F0AA2099F3F701858180FFA9C13E
:100F40008F708583ECCFAA2059F0093309F0B1C125
:100F5000FFEF17EE23E0F15010402040E1F7A7C16A
:100F6000812F0E942625A8C1812F869586958370A2
:100F700019F0813059F0A0C1DD2019F0C80193703B
:100F800002C080E090E00E949C1A9EC1DD2019F012
:100F9000C801937002C080E090E00E94861A94C15C
:100FA000812F837009F069C0D1108AC1902F92956A
:100FB00096959770990F990F802F8F70882E912C8E
:100FC000A12CB12C092E04C0880C991CAA1CBB1C96
:100FD0000A94D2F704FF12C04FE050E060E070E0E6
:100FE00004C0440F551F661F771F9A95D2F7DB0187
:100FF000CA0180959095A095B09503C080E090E0DF
:10100000DC0116951695412F4370423019F1C8F452
:1010100000916F0210917002209171023091720262
:10102000413059F088299929AA29BB29BC01CD0151
:1010300060237123822393230AC0802A912AA22A43
:10104000B32ABC01CD01682979298A299B290E94EC
:10105000112536C188299929AA29BB2900916F0237
:10106000109170022091710230917202BC01CD0189
:101070006027712782279327EACFDD2019F0812F7F
:10108000817001C08695882309F41AC1902F92952A
:1010900096959770990F990F802F8F70882E912CAD
:1010A000A12CB12C092E04C0880C991CAA1CBB1CB5
:1010B0000A94D2F704FF12C04FE050E060E070E005
:1010C00004C0440F551F661F771F9A95D2F7DB01A6
:1010D000CA0180959095A095B09503C080E090E0FE
:1010E000DC0116951695412F43704230D9F068F512
:1010F00000912C0210912D0220912E0230912F028E
:10110000413059F088299929AA29BB29BC01CD0170
:1011100060237123822393231EC0802A912AA22A4E
:10112000B32A13C088299929AA29BB2900912C0226
:1011300010912D0220912E0230912F02BC01CD0181
:10114000602771278227932706C0BC01CD0168293B
:1011500079298A299B290E948724B2C01F70DD202B
:1011600039F0812F0E94F024802F0E942D25A8C0E5
:10117000802F0E942625812F0E949124A1C0802FBC
:1011800032EF931609F443C0391538F090EF9916F1
:1011900059F0E1EF9E16B1F177C0F3EF9F16F1F130
:1011A00024EF921659F170C0DD2019F134E03A15A0
:1011B00008F482C01F7181E090E0A0E0B0E0AC01D3
:1011C000BD0104C0440F551F661F771F1A95D2F743
:1011D00080912C0290912D02A0912E02B0912F02AD
:1011E0008A019B01082719272A273B27C901B80133
:1011F00029C025E02A1508F45FC0DCCF80913102B8
:1012000082FF23C0DD2029F0812F8F7130C0DD20C7
:10121000D9F3812F8F710E9491244EC0DD2079F087
:101220001F7181E090E0A0E0B0E0BC01CD0104C0FE
:10123000660F771F881F991F1A95D2F703C060E0C9
:1012400070E0CB010E94872437C0DD2099F01F7128
:10125000812F0E94F0248091310282FD07C038E086
:10126000139FC0011124836080938203812F0E9409
:10127000F02422C081E00E94B62481E08A15E0F4C7
:1012800082E00E94B62418C0DD2029F0AA2009F4CB
:10129000BBCF802F14CEAA2009F4BBCF893349F4E9
:1012A0009FEFE7EEF3E09150E040F040E1F700C03F
:1012B0000000802F0E943C2888EF8B0D843020F4A2
:1012C0000E94B21A0E94B003CC20A9F08091820340
:1012D00080FD11C0F70112828595859585950E9444
:1012E000F024C7010E94CD038091820385958595E6
:1012F00085950E94912485E0F701DE011196019009
:101300000D928A95E1F789819A810E9430249A8111
:101310000CE6809FF001112419E0919FE00DF11D72
:1013200011248981E80FF11DEE0FFF1FE952FD4FD7
:1013300085919491F3C0023D8CE5180709F4DEC055
:1013400008F465C0053D8CE5180709F4DDC008F414
:1013500071C0063D2CE5120709F4DBC00E351D45B2
:1013600009F002CD80918203877009F4D7C0F7019C
:101370008281882309F4D2C08091310282FDCEC0DF
:1013800082E02A960FB6F894DEBF0FBECDBFDF9184
:10139000CF911F910F91FF90EF90DF90CF90BF9072
:1013A000AF909F908F900C94B62469E287CC053C57
:1013B000FCE51F0709F479C0063C1C4509F0D4CCB4
:1013C00047ED57E260EE77E28DC00A3C3CE513073B
:1013D00009F47AC070F4083CECE51E0709F46FC00C
:1013E000093C1C4509F0C0CC4BEC57E26FEB77E2AF
:1013F00079C00B3C2CE5120709F46BC00C3C1C4572
:1014000009F0B2CC4CE156E26DE276E26BC00F3CE3
:10141000ECE51E0709F46CC008F467C0003D2CE53C
:10142000120709F468C0013D1C4509F09DCC6EE02F
:1014300089E06CC0033DECE51E0709F462C0043D81
:101440001C4509F091CC61E088E165C08091CE0235
:1014500080FF20C08E7F8093CE026091CE0270917B
:10146000CF028091D0029091D1020E940A260E9460
:101470007F1C80919A02816080939A028FEF90E79F
:10148000E2E081509040E040E1F700C000000E949F
:10149000552568CF81608093CE0261E086953BC080
:1014A00049E258E262E378E21DC042E358E269E2B1
:1014B00078E218C040EE57E267ED77E213C04FEBD9
:1014C00057E26BEC77E20EC047EA57E263EB77E254
:1014D00009C043EB57E267EA77E204C04DE256E207
:1014E0006CE176E20E94791C3DCF61E081E013C09F
:1014F00065E082E00BC068E086E008C064E18FE050
:1015000005C067E185E102C062E289E10E94671CD3
:1015100029CF61E083E20E94E92724CF2A960FB603
:10152000F894DEBF0FBECDBFDF91CF911F910F9119
:10153000FF90EF90DF90CF90BF90AF909F908F90F3
:1015400008950F931F93CF93DF93CDB7DEB72897FE
:101550000FB6F894DEBF0FBECDBF85E0EEECF2E033
:10156000DE01119601900D928A95E1F78091980223
:1015700090919902A0919A028E839F83A88741E05F
:101580008885811101C040E008E010E09E012F5FD6
:101590003F4F69E072E086E00E94B0108111109226
:1015A0009A0228960FB6F894DEBF0FBECDBFDF912A
:1015B000CF911F910F9108950F931F93CF93DF93B6
:1015C0001F92CDB7DEB78091D30280FF04C086950D
:1015D0008695869501C080E0898341E09091F8016D
:1015E000981301C040E001E010E09E012F5F3F4FE3
:1015F00065E072E085E00E94B0100F90DF91CF911E
:101600001F910F910895CF93DF9300D000D0CDB7F5
:10161000DEB7409101025091020260910302709185
:1016200004022FB7F8948091DE029091DF02A0911E
:10163000E002B091E1022FBF841B950BA60BB70B04
:1016400084369105A105B10570F10E944811DC01B5
:10165000CB010296A11DB11D89839A83AB83BC8304
:1016600080912101909122018B519E4F4091200148
:1016700050E04530510510F044E050E0BE016F5F8E
:101680007F4F0E94E42B84E090E00E94762A88231A
:1016900059F00E941E1A6093010270930202809317
:1016A00003029093040281E00F900F900F900F902F
:1016B000DF91CF910895CF93DF93CDB7DEB72F970A
:1016C0000FB6F894DEBF0FBECDBF84B7877F84BF4F
:1016D0000FB6F894A89580916000886180936000AF
:1016E000109260000FBE90E080E80FB6F8948093EF
:1016F0006100909361000FBE85B7806885BF85B794
:10170000806885BF80E89FE09093E3018093E201C9
:101710000E94DE1F0E94FD1F8091E2008460809382
:10172000E20078948091F2028823A1F01091E90000
:101730001F709091EC00892F817090FD80E8182B2C
:101740001092E9008091E80083FD0E94CD1C1F707B
:101750001093E90082E084BD93E095BD9AEF97BDB8
:1017600080936E0010920E0210920F0210921002DF
:101770001092110287988F988FB1881F8827881F31
:101780008093470180914701882321F010926401E2
:1017900088E003C088E080936401809365010E9423
:1017A0000E1181110E948A2980914701811127C061
:1017B00086E0EAE6F1E0DE011A9601900D928A9544
:1017C000E1F7FE013A96A1E4B1E0CE0140969F0117
:1017D00041914D938E179F07D9F789E0E0E7F1E03B
:1017E000DE01119601900D928A95E1F7FE01319686
:1017F000A8E3B1E081918D932E173F07D9F780912F
:101800004701811102C096E001C090E090932B0245
:1018100086E0891B80932A0201E411E0A7E4EA2E06
:10182000A1E0FA2ED8018D918D018F3F11F00E9419
:101830003111E016F106B1F708E311E0F1E4EF2E03
:10184000F1E0FF2EF80181918F018F3F11F00E948E
:101850003111E016F106B1F788E1E4E3F2E0DF01CF
:10186000282F1D922A95E9F7E2E1F2E0DF011D92AF
:101870008A95E9F7269A80E090E00E94FF2A893E47
:101880009E4F11F00E945E1382E090E00E94F12AC8
:1018900080934C020E944D1390933102809330024A
:1018A0000E94D413EFE3FCE93197F1F700C0000088
:1018B0000E94D4138091340280FF08C06FEF7FEF45
:1018C00080E090E00E94232B0E94C51983E090E005
:1018D0000E94F12A682F70E080E090E00E941125BC
:1018E000259A2D9882E88093800089E18093810079
:1018F0008FEF9FEF90938700809386000E94391CA2
:101900000E94391C8091320281113BC080E090E03E
:101910000E94FF2A893E9E4F21F00E945E130E9482
:101920003E2688E090E00E94F92A6093CE027093F0
:10193000CF028093D0029093D10280919A0283606B
:1019400080939A026E7F71F40E943E2688E090E0B8
:101950000E94F92A6093CE027093CF028093D00246
:101960009093D1020E94F7250E947F1C8091CE02A5
:1019700080FF04C060E086950E94E92781E08093A3
:10198000320280914701811106C086E9809355019A
:1019900084E98093540180915501E82FE295EF701E
:1019A000F0E041A1282F2F7081E090E0BC0102C03F
:1019B000660F771F2A95E2F79B01362F3095342367
:1019C00031A332A1232B22A320915401E22FE295CF
:1019D000EF70F0E031A12F7001C0880F2A95EAF76F
:1019E000982F9095932391A392A1892B82A38FE89E
:1019F00091E00197F1F700C0000020915501E22F1E
:101A0000E295EF70F0E080A190E02F7002C0959514
:101A100087952A95E2F7817090915401E92FE2951C
:101A2000EF70F0E020A130E09F7002C0359527955F
:101A30009A95E2F720FD02C090E001C092E0892B68
:101A400080936C029091470181E0982790936B02FC
:101A5000891B809333020E940E11811102C00E94E3
:101A60008D2988E491E09093DA028093D90258E1BD
:101A7000C52ED12C60E4762E7CE4A72E72E0B72E22
:101A8000E0E16E2E8091F202853009F04BC012E148
:101A90008091F202853009F03DC08091F2028430DD
:101AA00039F180E00E944C1B80E00E94B00310924C
:101AB000DD020FB6F894A895C09260000FBE709238
:101AC000600083B7817F846083BF83B7816083BFF9
:101AD0007894889583B78E7F83BF0FB6F894A895C6
:101AE00080916000886180936000109260000FBE5A
:101AF0008091F102882309F4CBCF0E94D413E4E350
:101B0000F2E081919191892B09F0A3C1AE16BF0635
:101B1000C1F7BECF0E941B250E94391C0E94B21A39
:101B20000E94B0030E94D41381110E941E1AA4E3E4
:101B3000B2E0EDE4F2E000E010E0402E8D909D90E8
:101B400081919191882599250097A1F1512CEE243E
:101B5000E394F12C9C012E213F21232B29F10E949B
:101B60000E118823A9F059824A828E209F2081E09D
:101B7000892809F480E08B830E942A1A8160782FDB
:101B80009D838C8349815A816B818D810E940803DA
:101B9000000F111FF801E35BFD4F80819181E82662
:101BA000F926F182E0821CC05394EE0CFF1C29E060
:101BB0005212D0CF0F5F1F4F0C30110509F0BDCF6F
:101BC0008FEF8A878B871C860E942A1A8160782F64
:101BD0009E878D874A855B856C858E850E9408036C
:101BE0000E940E1180919902882309F4BDC0809152
:101BF0009802E091CE02E695E81BE09394028230D1
:101C000059F4F0E0EA51FF4FE4910E2F10E0ECECB4
:101C1000EE2EE8E1FE2E59C0863059F4F0E0ED5189
:101C2000FF4FE4910E2F10E07CEBE72E78E1F72ECA
:101C30004CC0893061F4E695F0E0E052FF4FE4914A
:101C40000E2F10E061E4E62E68E1F62E3EC08F30E4
:101C500061F4E695F0E0E352FF4FE4910E2F10E0BF
:101C60005CEAE52E57E1F52E30C0853159F4F0E0FD
:101C7000E652FF4FE4910E2F10E046E2E42E47E1DA
:101C8000F42E23C08831A1F0833249F4E8EDF0E06E
:101C9000059114913CE7E32E38E1F32E16C084320F
:101CA00071F404EF11E024E5E22E26E1F22E0DC0DE
:101CB00008E210E093E9E92E96E1F92E06C000ED66
:101CC00017E080EFE82E85E1F82E809195028823B9
:101CD00061F0109295020E94631190939302809399
:101CE000920210929702109296020E946311E09164
:101CF0009202F09193029C012E1B3F0B2F3F3F4716
:101D000098F5209167022223B1F01092670220918A
:101D1000650230916602821B930B8F3F9F4758F4F8
:101D2000205D3A48309366022093650280919A02C2
:101D3000886080939A0280909602909097020E0F8E
:101D40001F1F109393020093920282E992E0F70121
:101D500009958091960290919702892B29F4892800
:101D600019F081E080936702E0916C025E2F550FBD
:101D7000550F20915501E22FE295EF70F0E080A120
:101D800090E02F7002C0959587952A95E2F78170B3
:101D9000992740915401E42FE295EF70F0E020A1E3
:101DA00030E04F7002C0359527954A95E2F7F9016A
:101DB000E170FF2720FF02C0E2E0F0E0E82BF92B02
:101DC000E52BE0936C0210916B02EF70F0E0E558A8
:101DD000FE4F908180916A02890F80936A0284305D
:101DE0006CF0E12FF0E0E859FD4F80818F5F808338
:101DF00060E0812F0E94BA0321E001C020E08091C1
:101E00006A028D3F64F4E12FF0E0E859FD4F8081D4
:101E10008150808361E0812F0E94BA0321E080918C
:101E20006A02082E000C990B64E070E00E945D2BA2
:101E300080936A0221110E94F5120E94B21A9091B9
:101E40006D02891709F41ECE80936D020E94B003C3
:101E500019CE69BC19BD09B400FEFDCF8091D80030
:101E60008F7D8093D8008091E00082608093E000B5
:101E70008091E00081FDFCCF0E941B2509CEAF922E
:101E8000BF92CF92DF92EF92FF920F931F93CF9367
:101E9000DF937C015B016A0180910D028A3018F0AA
:101EA00001E010E002C00AE010E0C1E0D0E0F894E8
:101EB000B501C701F60109957894811115C02196E5
:101EC0000C171D0794F0CC9F9001CD9F300D300D65
:101ED000112480E090E045E34A95F1F70000019677
:101EE00082179307C1F7E3CF81E0DF91CF911F9174
:101EF0000F91FF90EF90DF90CF90BF90AF9008953B
:101F000080E008959091300292FF0DC0282F287133
:101F1000283019F4877F846006C0282F247124306C
:101F200011F48B7F886093FF0DC0282F2871283112
:101F300019F4877E846106C0282F2471243111F49E
:101F40008B7E88612091310220FF0DC0382F3871BF
:101F5000383019F4877F816006C0382F31713130F5
:101F600011F48E7F886021FF0DC0282F2871283141
:101F700019F4877E816106C0282F2171213111F467
:101F80008E7E886194FD877E08956F927F928F92F6
:101F90009F92AF92BF92CF92DF92EF92FF920F93F8
:101FA0001F93CF93DF931F92CDB7DEB7C62E4A01A2
:101FB0005901682E880F7708C3010E94762A88236A
:101FC00009F473C0C30123E0880F991F2A95E1F734
:101FD000FC01E050FF4F438150E04115510511F0E5
:101FE00041E050E0FC01E050FF4F648175816B518E
:101FF0007E4FCE0101960E94E42BF4014081518175
:10200000628173812FB7F8948091DE029091DF0294
:10201000A091E002B091E1022FBF841B950BA60BAB
:10202000B70B84369105A105B10538F4B701C80195
:102030000E94351B99818917D1F10C2C000CDD0809
:10204000C6010E94762A782E8823E1F0E114F1047B
:10205000C9F0960183E0220F331F8A95E1F7F90159
:10206000E050FF4F438150E0E416F50608F4A70165
:10207000F901E050FF4F648175816B517E4FC501BE
:102080000E94E42BB701C8010E94351B91E0298111
:10209000281390E0D92ED72089F00E941E1AF4014F
:1020A000608371838283938309C0D12C02C0DD24B5
:1020B000D394A701B801C5010E94E42B8D2D0F9088
:1020C000DF91CF911F910F91FF90EF90DF90CF9014
:1020D000BF90AF909F908F907F906F900895CF9218
:1020E000DF92EF92FF920F931F93CF93DF93CDB7C1
:1020F000DEB72C970FB6F894DEBF0FBECDBF6B01D5
:102100008CE0E82EF12C06EE11E09E012F5F3F4F90
:102110004AE852E061E080E00E94C50F882349F060
:102120009CE0FE013196AEE7B2E001900D929A95E7
:10213000E1F79CE0EEE7F2E0D60101900D929A956E
:10214000E1F72C960FB6F894DEBF0FBECDBFDF913E
:10215000CF911F910F91FF90EF90DF90CF90089556
:102160008F929F92AF92BF92CF92DF92EF92FF92A7
:102170000F931F93CF93DF93FB0180809180A28008
:10218000B3809FB7F894C090DE02D090DF02E09059
:10219000E002F090E1029FBFC818D908EA08FB08E6
:1021A000F4E6CF16D104E104F10410F4442341F124
:1021B0007B01C82F880FDD0B01151105A9F0FE0169
:1021C00083E0EE0FFF1F8A95E1F7E050FF4F81811A
:1021D00092818B519E4F408150E00417150708F4FF
:1021E000A801B9010E94E42BCE010E94762A88231F
:1021F00041F00E941E1AF7016083718382839383EA
:1022000081E0DF91CF911F910F91FF90EF90DF90D0
:10221000CF90BF90AF909F908F90089580917D0256
:10222000811118C08091D80080618093D8008AE124
:102230008A95F1F700C08091D90080FD02C082E04C
:1022400001C081E080937D02823021F40E94DE1F74
:102250001092F20281E090917D02913009F080E0CD
:102260000895F894E82FE295EF70F0E031A1282F5F
:102270002F7081E090E001C0880F2A95EAF7982F2F
:102280009095932391A392A1892B82A3789408958A
:102290000F931F930E940E11882321F01F910F911D
:1022A0000C941E1A0E941E1A00910E0210910F0229
:1022B0002091100230911102600F711F821F931F35
:1022C0001F910F9108950E940E1181110C942A1AEA
:1022D0000E944811CB010895CF93DF938238910576
:1022E00069F1B0F48133910509F46FC048F4893283
:1022F000910509F465C08A32910509F46BC08AC062
:102300008533910509F457C089339105B9F082C02E
:10231000833E910571F138F4803E9105B1F0823E23
:10232000910511F177C0863E9105B9F1873E91057F
:10233000C9F1843E910509F06DC024C0209130029E
:1023400020FD53C021FD51C065C08091300280FD49
:1023500046C08091310280FF48C08091300284FDE8
:102360003FC183EE90E03EC18091300282FF3AC0CF
:10237000F4CF8091300282FD35C08091310280FD22
:1023800034C0EBCF8091310281FF35C080913002A3
:1023900084FD26C187EE90E025C18091300283FF45
:1023A00027C0F4CF8091300283FD22C0809131029A
:1023B00081FD21C0EBCF8091300285FD1FC021C07F
:1023C0008091300285FD1DC019C08091300286FDCC
:1023D0001BC01DC08091300286FD19C015C089E365
:1023E00090E000C182EE90E0FDC080EE90E0FAC087
:1023F00086EE90E0F7C084EE90E0F4C089E290E0D1
:10240000F1C085E390E0EEC08AE290E0EBC081E3AA
:1024100090E0E8C0811532E5930708F069C08115A6
:1024200041E5940728F0982F8827816F906ADAC0D9
:10243000883E910568F5803E910508F0D3C0883A42
:102440009105B8F4853A910548F0855AE82FF0E0F7
:10245000E557FE4F808190E09064C4C081309105C3
:1024600009F4BBC008F4BCC08430910508F4B8C0BE
:10247000B9C08F3B910508F0B3C0885AE82FF0E04F
:10248000EE0FFF1FE257FE4F808191819464AAC036
:10249000811520E59207F0F09C0174E036952795B0
:1024A0007A95E1F7922F9370482F437021E030E046
:1024B00002C0220F331F4A95E2F73C68392B8F7018
:1024C000982F9695969540E2949FC0011124822BF7
:1024D000932B88C0811530E4930718F09F70906AA1
:1024E00081C09C013A9521153F4108F47BC078C01A
:1024F000EC01C11586E5D807E8F5C11525E5D20739
:1025000048F08C2F0E94820F8F7190E0982F8827BF
:10251000906268C0C11534E5D30728F09C2F882746
:10252000846F906A5FC0AE01437055272C2F2695AB
:102530002695C115D34578F481E090E002C0880F5C
:10254000991F4A95E2F740E2249F90011124822BC3
:10255000932B9C6847C081E090E002C0880F991FD0
:102560004A95E2F740E2249F90011124822B932B9D
:102570009A6838C0C1152AE5D207F8F4C11539E5C3
:10258000D30790F08C2F8F700E94820F94E0D69525
:10259000C7959A95E1F7CF70D0E0DC2FCC27D069B2
:1025A0009E01282BC9011EC0C11548E5D407C0F003
:1025B0009C2F8827806F906A15C0CE019056811598
:1025C000904270F48D2F8F710E94820F282F2F71EF
:1025D000CE0199279062922B05C081E090E002C065
:1025E00080E090E0DF91CF9108950C941E1ACF9275
:1025F000DF92EF92FF920F931F93CF93DF931F927F
:10260000CDB7DEB7EE24E394F12C03EF11E09E0189
:102610002F5F3F4F4EE852E063E082E00E94C50F1B
:10262000C82E882379F1D09033028D2D90E09C0143
:1026300028593D4F79011981F9018081181B012F1B
:1026400080E010165CF40150F70180818F5F808379
:1026500060E08D2D0E94BA0381E0F3CF912F17FD2A
:1026600090E0191B112359F01F5FF7018081815001
:10267000808361E08D2D0E94BA0381E0F3CF811148
:102680000E94F5128C2D0F90DF91CF911F910F9129
:10269000FF90EF90DF90CF900895CF9384E090E08B
:1026A0000E94F12AC82F82E290E00E94F12A2C2F8A
:1026B00030E0A901582BCA01CF91089569EE7EEF51
:1026C00080E090E00E94232B60E082E090E00E9496
:1026D000052B60E083E090E00E94052B10926F02D2
:1026E00010927002109271021092720260E084E007
:1026F00090E00E94052B60E082E290E00E94052BB2
:1027000060E085E090E00E94052B60E086E090E0CC
:102710000E94052B6FEF87E090E00E94052B40E0C0
:1027200050E0BA0188E090E00E94172B60E08DE055
:1027300090E00E94052B40E050E0BA0188E190E073
:102740000E94172B60E087E190E00E94052B40E09B
:1027500050E0BA018CE190E00E94172B60E070E03D
:1027600080E290E00E94232B40E050E0BA0188E133
:1027700090E00E94172B0E94211C83E00E94041C01
:1027800040E050E0BA018FE090E00E94172B40E05B
:1027900050E0BA0183E190E00C94172B80916E0217
:1027A000811110926E0208956F927F928F929F9284
:1027B000AF92BF92CF92DF92EF92FF920F931F934F
:1027C000CF93DF93CDB7DEB7A4970FB6F894DEBFF3
:1027D0000FBECDBF9E012F5F3F4F790188E1D90128
:1027E0001D928A95E9F701E411E0690167E4662E1C
:1027F00061E0762E88248394912CF80180818F3FAC
:1028000009F447C0F894E82FE295EF70F0E021A1B9
:102810008F70A40102C0440F551F8A95E2F7CA01C8
:10282000922F982B91A392A18095892382A37894CB
:1028300000C0E8E3F1E021E030E0A12CB12C4191AF
:102840004F3F89F0A42FA295AF70B0E090968C9185
:1028500090E04F7002C0959587954A95E2F780FD0C
:1028600002C0C90102C080E090E0A82AB92A220F64
:10287000331F51E0E134F50711F7D8018C918F3FF8
:1028800011F00E943111B0EABA95F1F7F601B18268
:10289000A0820F5F1F4FF2E0CF0ED11C60167106B1
:1028A00009F0ABCF48E150E0B70182E192E00E942D
:1028B000D72B8C01892B41F088E1F701A2E1B2E02E
:1028C00001900D928A95E1F7F0902B020115110508
:1028D00049F081E0809375020E942A1A9093740255
:1028E00080937302809175028823D9F080917302DE
:1028F000909174020E940F1A059798F0A2E1B2E03D
:10290000EF2DF0E0EE0FFF1FEC5CFD4F8EE192E04B
:102910002D913D91219331938A179B07C9F710920E
:1029200075020115110509F02CC10E940E11E091EC
:102930002B029E01275E3F4F7901882309F471C065
:102940008CE0D9011D928A95E9F70E2F10E0000F57
:10295000111F0C5C1D4F80910D028A3048F44FE628
:1029600050E1B701C8010E943F0F882359F10AC006
:1029700080917602909177020E940F1A843F9140D5
:1029800070F732C047EF52E1B701C8010E943F0F14
:102990008823C1F043E05BE0B701C8010E943F0F0C
:1029A000882381F04CED5AE0B701C8010E943F0F27
:1029B000882341F041EA5AE0B701C8010E943F0F65
:1029C0008111E2C080910D028F3F19F08F5F8093DB
:1029D0000D0280910D028A3008F4D8C00E942A1A94
:1029E000909377028093760280917C02811102C0DD
:1029F00000E0DFC08CE0F70111928A95E9F71092B0
:102A00007C02A0912A02B0E0AA0FBB1FAC5CBD4FB4
:102A10008CE0FE01799601900D928A95E1F701E034
:102A2000C8C0F894F0E0EE0FFF1FEC5CFD4F8CE0A7
:102A3000A6EEB1E001900D928A95E1F76CE070E0AE
:102A400086EE91E00E94351B8093E5017894F8941E
:102A5000E0916B02F0E0E859FD4F8081898F80930F
:102A6000F30161E070E0C7010E94351B8093F20121
:102A70007894F894C090F401D090F501E090F601BC
:102A8000F090F7018091780290917902A0917A02FA
:102A9000B0917B02C816D906EA06FB06D1F0C092B7
:102AA0007802D0927902E0927A02F0927B020E9440
:102AB0000E1181110EC00E941E1AC61AD70AE80A0A
:102AC000F90AC0920E02D0920F02E0921002F09228
:102AD00011027894F8948091F8010E944C1B78942C
:102AE000F89480910002882309F449C080FF24C033
:102AF0009091F9018091CE0290FF09C0816080938E
:102B0000CE0260E0892F86950E94E92715C08E7F4E
:102B10008093CE020E947F1C80919A0281608093F4
:102B20009A02FFEF20E732E0F15020403040E1F719
:102B300000C000000E9455258091000281FF09C05D
:102B400020E04091FC016091FB018091FA010E941C
:102B500005278091000282FF09C08091FF01882330
:102B600019F00E94861C02C00E947F1C8091000206
:102B700083FF03C081E08093950210920002789455
:102B800018C001E010E015C010920D0280912A02D9
:102B900090E0880F991F4CE050E0B7018C5C9D4F8E
:102BA0000E94D72B21E020937C02892B09F029CFAA
:102BB0001FCF802FA4960FB6F894DEBF0FBECDBFF7
:102BC000DF91CF911F910F91FF90EF90DF90CF9009
:102BD000BF90AF909F908F907F906F9008950895D1
:102BE000089508958091E70208958093E20270931A
:102BF000E4026093E3028091F202843001F582E006
:102C00008093E9008FEF9091E800815095FD06C018
:102C100095ED9A95F1F700008111F5CF8091E800CC
:102C200085FF0DC040E050E063E070E082EE92E08E
:102C30000E94A11C8091E8008E778093E80008959F
:102C4000BC0184E00C94F515BC0183E00C94F515EF
:102C5000CF93DF9321E02093E9002FEF3091E8003C
:102C6000215035FD06C035ED3A95F1F700002111F0
:102C7000F5CF2091E80025FF14C0EC0140E050E0C2
:102C800068E070E00E94A11C8091E8008E7780933C
:102C9000E80088E0FE01A8EEB2E001900D928A956E
:102CA000E1F7DF91CF9108950F931F93CF93DF93B7
:102CB000EC0100E010E080916801282F30E002175D
:102CC000130724F5909166019801290F311DA90180
:102CD000440F551F240F351F22563D4F869590E017
:102CE0004C81081719071CF4442331F002C041112C
:102CF00003C04091D10201C040E06091D0028091B8
:102D0000CF020E9455260F5F1F4FD5CF0E94552539
:102D10008C8190E00196817099278C83DF91CF910F
:102D20001F910F9108958F929F92AF92BF92CF9271
:102D3000DF92EF92FF920F931F93CF93DF938C015B
:102D4000FC014481C42FD0E09E01DE010E94A12B32
:102D50009B01AC010E94B72B6B017C01E0E2F0E02B
:102D6000EC1BFD0BA5E5B0E09B01AC010E94B72B6D
:102D70004B015C019F01DF010E94992B9B01AC017B
:102D80000E94C22B9B01AC012C0D3D1D4E1D5F1DF1
:102D9000C501B4010E94712BC22FD22F2A3228F410
:102DA000F3E02F9F900111240DC025E530E02C1B8E
:102DB0003109C901880F991F280F391F37FF02C039
:102DC0002F5F3F4F35952795C22FC095F12C85E594
:102DD000E82EED1A80916801F816C8F4F1FC02C0E3
:102DE0008E2D01C08D2F909166012F2D30E0290F7F
:102DF000311DA901440F551F240F351F22563D4F89
:102E00004C2F6091D0020E945526F394E3CF0E948C
:102E10005525F8018481811102C091E003C0803200
:102E200019F49FEF9093630190916301890FF8016A
:102E30008483DF91CF911F910F91FF90EF90DF90EE
:102E4000CF90BF90AF909F908F9008951F93CF9396
:102E5000DF93EC018C81811109C081E08C83109299
:102E60009C0292E0909362018093610180916601DF
:102E700090916701891770F4E82FF0E09F01220F0D
:102E8000331FE20FF31FE256FD4F118210821282B0
:102E90008F5FF0CF10E0609168011617C0F5E12F49
:102EA000F0E070E0CF010E945D2B20916601820F5F
:102EB00020919C02022E000C330B90E0E217F307E6
:102EC000CCF020916201022E000C330B2E173F072D
:102ED0008CF09C01220F331F820F931F9C012256FE
:102EE0003D4F4091D1026091D0028091CF020E946B
:102EF00055260BC0FC01EE0FFF1F8E0F9F1FFC011C
:102F0000E256FD4F1182108212821F5FC4CF0E94D1
:102F100055258091610120919C02280F20939C02ED
:102F200090916201980F9093620119165CF4022E41
:102F3000000C330B4091680150E0415051092417B7
:102F4000350734F0819580936101813009F41C824A
:102F5000DF91CF911F9108958F929F92AF92BF9270
:102F6000CF92DF92EF92FF920F931F93CF93DF9355
:102F7000EC018A8180FF03C0BB24BA9402C0BB2449
:102F8000B3948C8181110DC081E0B81206C080918C
:102F90006801815080939B0202C010929B0281E0E5
:102FA0008C83A12C90906801A91408F03EC08091F8
:102FB0006601CA2CD12C8601080F111DC801880F8B
:102FC000991F080F191F02561D4FF8011182108218
:102FD000128234E0E32EF12C812C80919B02880D2B
:102FE000813114F08F7002C087FD890D082E000C0E
:102FF000990BC816D90691F48091D1028E9DA0013B
:103000008F9D500D112455954795559547959801DD
:103010006091D0028091CF020E9455268B0CF1E086
:10302000EF1AF108D1F6A394BDCF0E9455258091E7
:103030009B0291E0B9120EC0811107C08091680116
:10304000815080939B021C820FC0815080939B0211
:10305000BC820AC090E001966091680170E00E9415
:103060005D2B80939B028C83DF91CF911F910F91F9
:10307000FF90EF90DF90CF90BF90AF909F908F9098
:103080000895FF920F931F93CF93DF93EC01F12CE0
:103090000FEF10E060916801F616F0F48091660180
:1030A0002F2D30E0280F311DC901880F991F280FDF
:1030B000391F22563D4F70E0C8010E945D2B962FAC
:1030C0008C814091D1026091D002F99E800D112433
:1030D0000E945526F394DECF0E9455259A818C815B
:1030E00090FF02C08F5F01C081508C83DF91CF9130
:1030F0001F910F91FF9008950F931F93CF93DF932C
:1031000000D01F92CDB7DEB78C0180919D02811156
:103110000AC09E012F5F3F4F4FEF6FEF0E94552671
:103120008A8180939D02F8018481813051F028F0DA
:10313000823061F440919D020AC080919D0240E07E
:1031400007C060919D0240E080E003C040E080E065
:1031500060E00E94DC25F801848190E0019663E044
:1031600070E00E945D2B84830F900F900F90DF9191
:10317000CF911F910F910895CF93DF93EC01EEEC67
:10318000F2E0438162818C810E94EB268C818F5F0B
:103190008C83DF91CF910895CF93DF93EC01EC8185
:1031A000F0E0E651FF4F4491EEECF2E06281818164
:1031B0000E94EB268C818F5F8C83DF91CF910895E5
:1031C0002091E4003091E50095E64091EC00842FD9
:1031D000817040FF23C08091E80080FD1DC0809178
:1031E000F202882399F0853099F08091EB0085FDFB
:1031F00011C04091E4005091E5002417350729F3F0
:10320000915011F09A01E1CF84E0089582E0089591
:1032100083E0089581E0089580E008954091E800FA
:1032200042FFDDCF08958091F40287FF11C08091A5
:10323000E80082FD05C08091F2028111F8CF11C033
:103240008091E8008B770BC08091F202882349F0CF
:103250008091E80080FFF8CF8091E8008E7780931E
:10326000E8000895982F973068F59093E900981733
:1032700039F07091EC002091ED005091F00003C006
:10328000242F762F50E021FD02C09F5FECCF3091BC
:10329000EB003E7F3093EB003091ED003D7F3093AB
:1032A000ED003091EB0031603093EB007093EC0057
:1032B0002093ED005093F0002091EE0027FDE5CF24
:1032C00080E008958F708093E90081E00895209157
:1032D000FA023091FB022617370748F06115710595
:1032E00039F42091E8002E772093E80001C0B9015D
:1032F000FC0120E06115710579F18091F2028823CB
:10330000F1F18530F1F18091E80083FD3CC08091BE
:10331000E80082FD2EC08091E80080FFEBCF209175
:10332000F3008091F20090E0922B6115710551F04D
:103330008830910538F421912093F1006150710992
:103340000196F3CF21E0089709F020E08091E80092
:103350008E778093E800CECF2111CFCF0AC0809125
:10336000F202882361F0853061F08091E80083FDEE
:103370000AC08091E80082FFF2CF80E0089582E0E9
:10338000089583E0089581E0089581E08093E0004E
:1033900080E28093D8001092C9008FE19EE40197EB
:1033A000F1F700C0000087E090EBDC0180938D0313
:1033B00090938E03A0938F03B09390039CE088E1D9
:1033C0000FB6F894A895809360000FBE90936000AC
:1033D000FFCF78941F920F920FB60F9211248F9304
:1033E0009F93AF93BF938091DE029091DF02A091F3
:1033F000E002B091E1020196A11DB11D8093DE02B1
:103400009093DF02A093E002B093E102BF91AF91ED
:103410009F918F910F900FBE0F901F9018959C0158
:103420004FB7F8948091DE029091DF02A091E00204
:10343000B091E1024FBF821B930B08952FB7F89410
:103440006091DE027091DF028091E0029091E102D2
:103450002FBF08952FB7F8948091DE029091DF027C
:10346000A091E002B091E1022FBF08951F920F9248
:103470000FB60F9211248F939F93AF93BF938091B8
:10348000DD02811113C08091DE029091DF02A091D4
:10349000E002B091E1024196A11DB11D8093DE02D0
:1034A0009093DF02A093E002B093E102BF91AF914D
:1034B0009F918F910F900FBE0F901F9018959C01B8
:1034C0002A5F3F4FFC014281461301C012820196E0
:1034D00082179307B9F708959C01FC0132969FEF7C
:1034E00080E04191461789F09F3F19F4411101C0D6
:1034F000982F8F5F8630A9F79F3F39F0F901E90FC8
:10350000F11D97FDFA956283089508952091DB02DD
:103510003091DC022817390771F09093DC02809318
:10352000DB02E091D902F091DA02309721F00084B9
:10353000F185E02D099408952091D7023091D802A9
:103540002817390771F09093D8028093D702E09141
:10355000D902F091DA02309721F00680F781E02D50
:10356000099408950E940E11882351F0E091D90228
:10357000F091DA02309721F00190F081E02D09946A
:1035800080E008950F931F93CF93DF93C42FD22F22
:10359000FC0182818823C9F04093D6020E942A1A36
:1035A0009093D5028093D40280E28C0F883008F08B
:1035B00057C0C77081E001C0880FCA95EAF7DF9154
:1035C000CF911F910F910C942D258091D602481315
:1035D00030C08091D4029091D5020E940F1A883C8D
:1035E000910538F510E21D0FCD17B9F080E28C0F70
:1035F000883040F4C77081E001C0880FCA95EAF7AF
:103600000E942625183028F581E09D2F977001C073
:10361000880F9A95EAF70E942D25802F0E94372562
:103620001830F0F4D77081E001C0880FDA95EAF71E
:103630000AC080E28C0F883098F4C77081E001C026
:10364000880FCA95EAF7DF91CF911F910F910C94E3
:103650002625802FDF91CF911F910F910C94372554
:10366000DF91CF911F910F910895FC01680F791F91
:103670008FEF91E3E617F70771F02191822728E099
:1036800030E087FF03C0880F892701C0880F2150D1
:103690003109B9F7EFCF08958F929F92AF92BF9201
:1036A000CF92DF92EF92FF920F931F93CF93DF930E
:1036B000843048F4811108C0909180009F779093E6
:1036C00080002D9806C083E09091800090689093D0
:1036D0008000A0918600B0918700282F30E00E94E2
:1036E000A12B23E030E040E050E00E94712B002746
:1036F000122F232F342F012F122F232F33278091A6
:103700008600909187006CE070E00E94492B601762
:10371000710730F0C80169E070E00E94492B5EC07B
:103720008091860090918700E0908600F09087005D
:10373000E0918600F0918700C6E0D0E0BE010E94D3
:10374000492B060F171F211D311D4801590185E026
:10375000880C991CAA1CBB1C8A95D1F7C701BE0115
:103760000E94492B6F01E12CF12CA7019601260F35
:10377000371F411D511DC501B4010E94712B690104
:103780007A01E0918600F0918700CA01B9010E9498
:10379000392B9B01AC01DF010E94B72B9B01AC01CF
:1037A000C701B6010E94392BDC01CB012FE0B69591
:1037B000A795979587952A95D1F700918600109146
:1037C000870020E030E0081719072A073B0728F494
:1037D0006091860070918700CB01BC0170938900D5
:1037E00060938800DF91CF911F910F91FF90EF9030
:1037F000DF90CF90BF90AF909F908F900895682FEB
:1038000086E090E00C94052B843008F083E09091E2
:10381000D3029770282F220F220F220F922B909302
:10382000D302987F21E009F420E09091D30220FB9D
:1038300090F99093D3020E944C1B8091D3020C9478
:10384000FF1B8091D30280FD13C081608093D3025F
:10385000813019F489E08093D3028091D3020E94D1
:10386000FF1B8091D3028695869586950C944C1B00
:10387000089580E090E00E94FF2A893E9E4F51F01B
:103880000E945E138091D302847089618093D30279
:103890000E94FF1B86E090E00E94F12A8093D302F1
:1038A000282F26952695269530E02430310524F0E2
:1038B000877088618093D3028091D30280FF04C017
:1038C00086958695869501C080E00C944C1B90915E
:1038D000CE0290FF04C09695981740F003C0811166
:1038E00005C090E0961710F40C94322861E00C9417
:1038F000E927882311F0FA0101C0FB010994E8E9E6
:10390000F2E0118282818460828308956091CE0208
:10391000669570E04BE050E086E591E00E94CA2B8E
:10392000892B19F481E0809399020E94631190938E
:1039300093028093920280919A02846080939A020B
:103940000895EF92FF920F931F93CF93DF937C0123
:103950008B010E94E018811119C0E70101151105C2
:10396000A1F08091E80085FD0AC08091E8008E7783
:103970008093E8000E94E018882381F307C08991B2
:103980008093F10001501109E9CF80E0DF91CF91E0
:103990001F910F91FF90EF9008951F93CF93DF93A6
:1039A000CDB7DEB7AA970FB6F894DEBF0FBECDBF76
:1039B000E4EFF2E08CEF92E02091F10021938E177A
:1039C0009F07D1F78091F502833009F461C030F48C
:1039D000813071F0823009F49BC0B2C08A3009F4A2
:1039E00087C08B3009F46CC0893009F0A9C020C0B1
:1039F0008091F402813A09F0A3C08091E800877FAA
:103A00008093E8008091F8029091F902892B21F4CB
:103A100068E088EE92E003C060E080E090E070E053
:103A20000E9467198091E8008B778093E80088C036
:103A30008091F402813209F083C08091F802909164
:103A4000F902029708F07CC08091E800877F80939C
:103A5000E8008091E80082FD05C08091F2028111AA
:103A6000F8CF6EC02091F3008091F20090E0922B8D
:103A7000029731F48091F100813011F0863021F409
:103A80008091F1008093E7028091E8008B7754C029
:103A90008091F402813A09F053C08091F80290912C
:103AA000F902892B09F04CC08091E800877F809350
:103AB000E8008091E80080FFFCCF8091690137C069
:103AC0008091F4028132E1F58091F8029091F9023F
:103AD000892BB1F58091E800877F8093E8000E94F0
:103AE00013198091F602809369010E941B2528C05A
:103AF0008091F402813221F58091E800877F8093E4
:103B0000E8000E9413198091F7028093E60218C022
:103B10008091F402813AA1F48091E800877F80933C
:103B2000E8008091E80080FFFCCF8091E60280935E
:103B3000F1008091E8008E778093E8000E941319CD
:103B40008091E80083FFCEC18091F4029091F5024C
:103B5000492F50E04A30510508F0C4C1FA01EE592E
:103B6000FF4F0C94932B803821F0823809F0BAC1B2
:103B700008C08091F0029091F102992389F082604F
:103B80000FC08091F8028F70873008F0ABC180932E
:103B9000E9008091EB0085FB882780F91092E9000D
:103BA0009091E800977F9093E8008093F100109245
:103BB000F10065C1282F2D7F09F094C1882319F0E9
:103BC000823061F08FC18091F602813009F08AC1A4
:103BD000933009F080E08093F1022EC08091F602CC
:103BE00081112AC08091F8028F702FEF280F2630A4
:103BF00008F078C18093E9002091EB0020FF1CC001
:103C0000933021F48091EB00806214C09091EB001E
:103C100090619093EB0021E030E0A90102C0440FD5
:103C2000551F8A95E2F74093EA001092EA008091CE
:103C3000EB0088608093EB001092E9008091E8002F
:103C4000877F20C181114EC11091F6021F778091AC
:103C5000E3008078812B8093E3008091E800877FE8
:103C60008093E8000E9413198091E80080FFFCCF48
:103C70008091E30080688093E300111102C082E02C
:103C800001C083E08093F2022DC18058823008F099
:103C900029C18091F6029091F7028C3D53E095077F
:103CA00079F583E08A838AE289834FB7F894DE014D
:103CB000139620E03EE051E2E32FF0E050935700EE
:103CC000E49120FF03C0E295EF703F5FEF708E2F0D
:103CD00090E0EA3010F0C79601C0C0968D939D9396
:103CE0002F5F243149F74FBF8091E800877F809391
:103CF000E8006AE270E0CE0101960E946719AEC04A
:103D00004091F8025091F902292F332723303105D1
:103D1000A9F068F42130310509F4F3C022303105EF
:103D200009F0E0C08BE390E0ECE5F2E044C0213222
:103D3000310521F12232310571F1D4C0992781304A
:103D40009105A1F058F0029709F0CCC0E9EAF2E041
:103D5000E4918E2F90E0E9EAF2E02AC0E3EDF2E090
:103D6000E4918E2F90E0E3EDF2E022C0E3ECF2E08C
:103D7000E4918E2F90E0E3ECF2E01AC0411551057A
:103D800009F4C4C04130510509F0ACC089E090E0AD
:103D9000E7E8F2E010C04115510509F4BCC041301C
:103DA000510509F09FC082E390E0EAEEF1E003C024
:103DB000009709F497C02091E800277F2093E8003E
:103DC0002091FA023091FB028217930708F49C01BC
:103DD00040E02115310589F18091F202882309F430
:103DE0003DC08530D9F18091E80083FD37C08091D6
:103DF000E80082FD2FC08091E80080FFEACF40916B
:103E0000F3008091F20090E0942B2115310559F0D8
:103E10008830910540F444914093F100319621504F
:103E200031090196F2CF41E0089709F040E0809116
:103E3000E8008E778093E800CCCF4111CDCF0AC047
:103E40008091F202882351F0853041F08091E800A2
:103E500083FD04C08091E80082FFF2CF8091E800EA
:103E60008B778093E8003EC08038E1F58091E800D0
:103E7000877F8093E8008091F3028093F100809126
:103E8000E8008E778093E8000E9413192BC08111FF
:103E900029C08091F6029091F7029927029714F5B4
:103EA0008091E800877F8093E8001091F6021093DC
:103EB000F3020E941319111106C08091E30087FDDF
:103EC00002C081E001C084E08093F20242E061EC34
:103ED00081E00E94321942E261EC82E00E943219D4
:103EE0008091F2028091E80083FF1AC08091E8007F
:103EF000877F8093E8008091EB0080628093EB00E5
:103F00000FC082E190E0E7E9F2E055CF89E090E070
:103F1000EEE6F2E050CF80E490E0ECE1F2E04BCF4F
:103F2000AA960FB6F894DEBF0FBECDBFDF91CF913A
:103F30001F9108951F920F920FB60F9211242F9385
:103F40003F934F935F936F937F938F939F93AF9321
:103F5000BF93CF93DF93EF93FF93C091E900CF70AE
:103F60008091EC00D82FD17080FDD0E81092E9004C
:103F70008091F000877F8093F00078940E94CD1CA0
:103F80001092E9008091F00088608093F000CD2BC2
:103F9000CF70C093E900FF91EF91DF91CF91BF9176
:103FA000AF919F918F917F916F915F914F913F91D1
:103FB0002F910F900FBE0F901F901895E8EDF0E035
:103FC00080818E7F80831092E2001092DA0010923E
:103FD000E100A0EEB0E08C9181608C9380818F77BE
:103FE000808319BCA7EDB0E08C918E7F8C9380818B
:103FF0008F7E80831092E5020895CF92DF92EF9238
:10400000FF920F931F93CF93DF93C8EDD0E0888189
:104010008F7E8883E7EDF0E080818160808384E09B
:1040200082BF81E08093E50288818E7F888302EEE3
:1040300010E0F80110821092DA0081EEC82ED12C27
:10404000F601108288818F778883888180688883D1
:1040500088818F7D888319BC1092F2021092F3023E
:104060001092F1021092F00290EEE92EF12CF7017D
:1040700080818B7F808388818160888342E060E0DB
:1040800080E00E943219F60180818E7F8083F801E2
:10409000808181608083808188608083F701808156
:1040A0008E7F8083888180618883DF91CF911F918B
:1040B0000F91FF90EF90DF90CF9008951F920F9295
:1040C0000FB60F9211242F933F934F935F936F93EB
:1040D0007F938F939F93AF93BF93EF93FF938091C1
:1040E000E10082FF09C08091E20082FF05C080915B
:1040F000E1008B7F8093E1008091DA0080FF2AC08D
:104100008091D80080FF26C08091DA008E7F809356
:10411000DA008091D90080FF18C080E189BD82E17A
:1041200089BD09B400FEFDCF81E08093F202809149
:10413000E50281110FC00E94DE1F0E94FD1F8091C9
:10414000E20084608093E20005C019BC1092F20284
:104150001092E5028091E10080FF17C08091E2009B
:1041600080FF13C08091E2008E7F8093E2008091F7
:10417000E20080618093E2008091D80080628093A9
:10418000D80019BC85E08093F2028091E10084FFA1
:1041900030C08091E20084FF2CC080E189BD82E1C3
:1041A00089BD09B400FEFDCF8091D8008F7D80933A
:1041B000D8008091E1008F7E8093E1008091E20041
:1041C0008F7E8093E2008091E20081608093E20024
:1041D0008091F302882311F084E007C08091E3000E
:1041E00087FD02C081E001C083E08093F2028091EC
:1041F000F2028091E10083FF27C08091E20083FFFB
:1042000023C08091E100877F8093E10082E080936A
:10421000F2021092F3028091E1008E7F8093E10020
:104220008091E2008E7F8093E2008091E2008061C5
:104230008093E20042E060E080E00E9432198091C9
:10424000F00088608093F000FF91EF91BF91AF91F3
:104250009F918F917F916F915F914F913F912F919E
:104260000F900FBE0F901F901895809590918C0322
:10427000892380938C03089590918C0380918B0304
:10428000982B9093FC0280916E02882389F0892BF1
:104290008093FC02EEEFF2E097E080E0915029F08D
:1042A00021912223D9F38F5FF9CF81110E94CE1380
:1042B00048E050E063E873E08CEF92E00E94D72B77
:1042C000892BA9F088E0ECEFF2E0A3E8B3E00190DD
:1042D0000D928A95E1F7E091D902F091DA023097D8
:1042E00031F00280F381E02D8CEF92E00994089583
:1042F00080E090E00E949C1A80E090E00E94861A84
:1043000010928B030C943C21809181039091500377
:10431000891719F08F5F8770FBCF08950F931F9354
:10432000CF93DF9380914F0382958F7009F05DC02A
:1043300080914C03882309F458C080918103109127
:10434000500360914A0370914B03C0914D03D0918B
:104350004E0391E06F3F09F090E0292F06E08117AE
:1043600009F443C0209721F07F3F21F030E003C0E3
:1043700031E001C0322F90E030FD34C0089FF001E1
:10438000099FF00D1124DF01AF5ABC4F11963C91EB
:104390001197371327C03C91361324C012963C91D5
:1043A000129731111FC013964D915C9114974C1BBD
:1043B0005D0B483C5105B0F480914F038F708061D4
:1043C00080934F03EA5AFC4F80818F708061808315
:1043D0008AE493E00E94CD03DF91CF911F910F916A
:1043E0000C94842101968770BACFDF91CF911F91F1
:1043F0000F9108958F929F92AF92BF92DF92EF92AA
:10440000FF920F931F93CF93DF9380902C02909095
:104410002D02A0902E02B0902F0240916F02509179
:1044200070026091710270917202842A952AA62A04
:10443000B72ACFE1D0E029E0929F700111249CE6D9
:10444000D92E082F10E0D501C4010C2E04C0B6955A
:10445000A795979587950A94D2F780FD04C0219778
:1044600090F780E014C0DC9EF001DD9EF00D112479
:10447000EE0DFF1DE00FF11FEE0FFF1FE952FD4F84
:10448000859194910E946C11019749F38C2FDF91D3
:10449000CF911F910F91FF90EF90DF90BF90AF9061
:1044A0009F908F900895CF93DF93EC010E94FA21A3
:1044B0002CE6829FC0011124FC0129E0D29FE00D6F
:1044C000F11D1124EC0FF11DEE0FFF1FE952FD4FFE
:1044D000859194910E946C11DF91CF910895FC0118
:1044E000808191810E94532292959F70963079F03D
:1044F00010F4925001C09A50923068F4803F69F0F5
:1045000018F4883E40F409C0843F29F406C0883E70
:1045100020F0813F11F080E0089581E008959F929E
:10452000AF92BF92CF92DF92EF92FF920F931F93C1
:10453000CF93DF93CDB7DEB761970FB6F894DEBFA8
:104540000FBECDBF8C0185E0F801DE011D96019004
:104550000D928A95E1F7F801E28090914A0360910B
:104560004B0340914D0350914E034115510531F0DD
:104570006F3F31F481E09F3F19F403C081E001C037
:1045800080E0F82FF1709F2E80FD1AC1F801308174
:104590002181C380D4808AE4A82E83E0B82EF090D5
:1045A0004C03F601E41BF50BFF2009F4C6C0809113
:1045B0004F03E83CF10508F091C0482F407F09F017
:1045C00050C0621311C093130FC0FE2CE1100CC039
:1045D0008F70806180934F03C5010E94CD0380914D
:1045E0004F03F801858329C1CD2831F02F3F31F4E5
:1045F00081E03F3F19F403C081E001C080E080FD0D
:1046000003C081E08E2502C080E090E0F82FF170B9
:10461000FF2E80FF1CC0809181034091500356E023
:10462000841709F4E8C090E0589FF001599FF00DFD
:104630001124EF5AFC4F6181261306C06081631379
:1046400003C06281E61203C001968770E9CFFE2C99
:10465000EE2009F4F2C080914F03816080934F03F4
:1046600049C0621306C0931304C0E11002C0F801F0
:1046700086C0C8010E946F22882351F1EE2041F1CB
:1046800020914F03822F82958F7090E0029774F0F3
:1046900080914A0390914B0398878F831986DB861C
:1046A000CA862C87CE0107960E94CD0386E0F801CA
:1046B000AAE4B3E001900D928A95E1F70E948E2161
:1046C0000AC06217C9F0C8010E946F2281111EC082
:1046D000C8010E94CD03FF24F394AFC0482F407F50
:1046E00081F78AE493E00E94CD0386E0F501119200
:1046F0008A95E9F7F12CA1C09313E5CFE110E3CF40
:10470000F8018583C8010E94CD0354C0EE2001F357
:1047100020914F03822F82958F7090E0029734F2A0
:1047200080914A0390914B039A8389831B82DD8297
:10473000CC822E83CE010196B7CFE83CF105D0F5AF
:10474000FE2CEE2029F2621327C0931325C020917E
:104750004F0320FD18C0822F82958F70482F50E0A4
:104760004115510581F0F80125834F30510541F085
:104770008F5F982F9295907F822F8F70892B8583E2
:10478000C8010E94CD0386E0F801AAE4B3E00190DD
:104790000D928A95E1F751C0C8010E946F228111E4
:1047A00085CF80914F03816080934F03C8010E94A1
:1047B000CD0343C086E0F50111928A95E9F73DC02B
:1047C000EE2009F485CFC8010E946F22F82E8823BD
:1047D00009F47ECF86E0F801AAE4B3E001900D92DF
:1047E0008A95E1F780914A0390914B030E945322EE
:1047F0000E948E2122C03D872E878D859E850E9436
:104800005322292F22952F70223028F49F7039F0DF
:10481000811105C00BC0243028F49F7049F4805EDC
:10482000883020F0C8010E94CD039F2CF92C05C0D0
:10483000F8019581907F99F7F9CF8F2D61960FB68A
:10484000F894DEBF0FBECDBFDF91CF911F910F91C6
:10485000FF90EF90DF90CF90BF90AF909F90089522
:1048600029E0929F800D1124682F669566956695C4
:10487000982F977085E0689FB001112440E050E0C8
:1048800080E0FB01E40FF51FEC5FFC4F208130E07E
:10489000092E02C0369527950A94E2F72170332736
:1048A000042E01C0220F0A94EAF7822B4F5F5F4F5C
:1048B0004530510531F7089529E0929F800D11246C
:1048C000E82FE695E695E695877051E001C0550F13
:1048D0008A95EAF785E0E89FF0011124EC5FFC4F30
:1048E00020E030E070E04081CB01022E02C09695BE
:1048F00087950A94E2F78170819584278523842720
:1049000081932F5F3F4F2530310569F708956093FC
:104910002C0270932D0280932E0290932F020C9400
:1049200078210F931F9341E050E060E070E004C0F5
:10493000440F551F661F771F8A95D2F740955095F3
:104940006095709580912C0290912D02A0912E027D
:10495000B0912F028A019B01082319232A233B23AC
:10496000C901B8011F910F910C94872420918203F3
:104970008095822380938203982F977099F430E07A
:10498000482F082E000C550B2417350759F090912D
:10499000310292FD07C08595859585950E949124E9
:1049A000109282030895CF93C0913102C2FB9927E0
:1049B00090F9981799F080FBC2F9C0933102609189
:1049C000300284E090E00E94052B6C2F82E290E0A0
:1049D0000E94052B82E0CF910C94B624CF910895CC
:1049E0000F931F9341E050E060E070E004C0440F7B
:1049F000551F661F771F8A95D2F780912C029091E0
:104A00002D02A0912E02B0912F028A019B01082B4A
:104A1000192B2A2B3B2BC901B8011F910F910C9424
:104A2000872460936F027093700280937102909359
:104A300072020C94782110928C0386E0EEEFF2E083
:104A4000DF011D928A95E9F70C947821882321F0E3
:104A50000E9435210C943C210895882339F09091CF
:104A60008C03892B80938C030C943C2108951F9315
:104A7000CF93DF93182F893319F0C0E0D0E002C044
:104A8000C0E5D0E0812F0E949328209741F08FE964
:104A90009FE00197F1F700C000002197F6CF812F2A
:104AA000DF91CF911F910C943C28CF92DF92EF922F
:104AB0000F931F93CF93DF93CDB7DEB7E0970FB679
:104AC000F894DEBF0FBECDBF609165018091CE022C
:104AD00080FF0AC0ECE8F5E0AE014F5F5F4F8E014A
:104AE0000F5C1F4FCA0114C080916601909167014D
:104AF000891780F7E82FF0E09F01220F331FE20FA4
:104B0000F31FE256FD4F1182108212828F5FF0CFA9
:104B1000249130E0D901AA0FBB1F2A0F3B1FD901F6
:104B2000A256BD4FCD90DD90EC90DA01CD92DD9292
:104B3000ED92AD013196A017B10751F720916401B4
:104B4000FC01B3E02B9FE00DF11D11246E9A8EB194
:104B50008F7B9EB190642FB7F894AF0133E0639FD1
:104B6000400D511D1124E417F50789F0319168E0DB
:104B70009EB9000000C037FF8EB9330F000000C09F
:104B800000C000C08EB900C06A9591F7ECCF2FBF6E
:104B90008FE594E00197F1F700C00000E0960FB6B2
:104BA000F894DEBF0FBECDBFDF91CF911F910F9163
:104BB000EF90DF90CF9008959091CE0290FF16C0B5
:104BC0009091660120916701921770F4E92FF0E04F
:104BD000DF01AA0FBB1FEA0FFB1FE256FD4F8183C7
:104BE000608342839F5FF0CF0C9455250895809198
:104BF000CE02282F269530E02115310519F4817059
:104C0000826005C02532310524F08170886480936C
:104C1000CE020895CF92DF92EF92FF926B017C015A
:104C20000E94F725B701A60188E090E0FF90EF9081
:104C3000DF90CF900C94172B8091D202882319F02B
:104C400081508093D2026091CE027091CF02809108
:104C5000D0029091D1020C940A268091D202833026
:104C600018F48F5F8093D2026091CE027091CF02D0
:104C70008091D0029091D1020C940A26EEECF2E0E1
:104C800087E1808311828FEF828383831482A8E976
:104C9000B2E012968C911297836012968C93608189
:104CA0007181828193810C940A26AF92BF92CF9238
:104CB000DF92EF92FF920F931F93CF93DF93E82E33
:104CC000F62EE901E42FF0E0611106C0E957FB4F31
:104CD000E4914E2F2E2F71C0062F10E0E957FB4FA5
:104CE0004491F42FC42ED12C26E0829FC0011124C0
:104CF0002FEF30E0B9010E94492B5BEA5603C00157
:104D0000579F900D11248E0D911D8E0D911D582FC2
:104D1000550F580FD901A01BB10BAC9DC001AD9D23
:104D2000900DBC9D900D1124E92FF59ED00111240A
:104D3000AB2FBB277901EA1AFB0AEC9CD001ED9C52
:104D4000B00DFC9CB00D11245901A51AB108A09E0C
:104D50007001A19EF00CB09EF00C1124EF2CFF24EA
:104D60002E193F092C9D80012D9D100D3C9D100D8D
:104D70001124212F6230710591F048F461157105FD
:104D8000E1F061307105B9F4242F4B2F16C0643067
:104D9000710569F040F06630710579F00CC0242F80
:104DA000492FE12F0AC0492FEF2F2B2F06C0292FA3
:104DB000E42F412F02C0292FEB2F49832883EA8358
:104DC000DF91CF911F910F91FF90EF90DF90CF90E7
:104DD000BF90AF900895CF93DF9300D01F92CDB7CF
:104DE000DEB79091CE0290FF0AC09E012F5F3F4F29
:104DF0000E9455264B8169818A810E94DC250F9093
:104E00000F900F90DF91CF910895AF92BF92CF9204
:104E1000DF92EF92FF920F931F93CF93DF9300D017
:104E20001F92CDB7DEB7182FF62E042FE22E9091E9
:104E3000CE0290FF7EC0E92FE695AE2FB0E0A454DD
:104E4000BE4F8C91809398029E7F923061F49E01B8
:104E50002F5F3F4F812F0E9455264B8169818A81A8
:104E60000E94DC2543C0823019F40091D1023EC07B
:104E7000863019F41091CF0239C08930D9F38931C5
:104E8000A9F5E9518E2F8170D82EE695F0E0E9570B
:104E9000FA4FA590B490C12CBB2460916801C6164E
:104EA00018F52C2D30E0A29EC001A39E900DB29E5D
:104EB000900D112470E00E94492B812FD11002C067
:104EC000860F01C0861B90916601290F311DA90133
:104ED000440F551F240F351F22563D4F402F6F2D75
:104EE0000E945526C394D9CF0E9455258091CF02A8
:104EF000181308C08091D002F81204C08091D1022A
:104F0000081729F080919A02826080939A02109388
:104F1000CF02F092D0020093D102EE2051F06091C6
:104F2000CE027091CF028091D0029091D1020E9466
:104F30000A260F900F900F90DF91CF911F910F9144
:104F4000FF90EF90DF90CF90BF90AF900895EEEC80
:104F5000F2E0438121E1421B08F440E021E062815C
:104F600081810C940527EEECF2E0438121E1420FB0
:104F700008F44FEF21E0628181810C940527EEEC6B
:104F8000F2E0628121E1621B08F460E021E04381EC
:104F900081810C940527EEECF2E0628121E1620F41
:104FA00008F46FEF21E0438181810C940527EEEC3A
:104FB000F2E0818121E04381628188500C940527D1
:104FC000EEECF2E0818121E043816281885F0C9404
:104FD00005279091CE0290FF3BC09170811102C0D5
:104FE000926006C0853210F0986402C0880F982B3A
:104FF0009093CE0280919A02816080939A026623F8
:1050000051F06091CE027091CF028091D0029091C8
:10501000D1020E940A266091CE02669570E04BE0B4
:1050200050E086E591E00E94CA2B892B19F00E947E
:105030007F1C02C00E94861C81E08093950220E0C4
:105040004091D1026091D0028091CF020C9405274B
:1050500008958091CE028695815009F484E261E042
:105060000C94E9278091CE0286958F5F853208F0F7
:1050700081E061E00C94E927882309F453C0682F8C
:10508000823869F40E94B21A81FF4CC069E38CEF48
:1050900092E00E946C1A0E943C2169E30EC08338A2
:1050A00091F40E94B21A80FF3DC063E58CEF92E05C
:1050B0000E946C1A0E943C2163E58CEF92E00E94F2
:1050C0005F1A0C943C21843869F40E94B21A82FF62
:1050D00029C067E48CEF92E00E946C1A0E943C2188
:1050E00067E4EBCF8CEF860F813A38F380E2860FCE
:1050F000883048F4677081E001C0880F6A95EAF74C
:105100000E943521DECF8BE5860F833020F480E0CE
:1051100090E00C949C1A685A673120F480E090E08B
:105120000C94861A0895CF93882309F496C0C82F4B
:105130008238B1F40E94B21A81FD8FC069E38CEF0E
:1051400092E00E946C1A0E943C212FEF81EE94E0C5
:10515000215080409040E1F700C0000069E317C093
:105160008338E1F40E94B21A80FD77C063E58CEFCA
:1051700092E00E946C1A0E943C212FEF81EE94E095
:10518000215080409040E1F700C0000063E58CEFC3
:1051900092E00E945F1ACF910C943C218438B1F4C4
:1051A0000E94B21A82FD59C067E48CEF92E00E941F
:1051B0006C1A0E943C212FEF81EE94E02150804038
:1051C0009040E1F700C0000067E4E1CF8CEF8C0F66
:1051D000813A80F4EEEFF2E084E093E02191C2178F
:1051E000A1F18E179F07D1F76C2F8CEF92E00E94F0
:1051F0006C1AD1CF80E28C0F883068F4C77081E0E0
:1052000090E001C0880FCA95EAF790918C03892B32
:1052100080938C03C0CFEBE5EC0FE33040F4F0E07B
:10522000E557FE4F808190E0CF910C949C1AC85AAC
:10523000C73198F4EC2FF0E0EE0FFF1FE257FE4F5E
:1052400080819181CF910C94861A6C2F8CEF92E023
:105250000E945F1A0E943C21C7CFCF9108958EE132
:10526000489B02C08150E1F7489BFECF08955898B3
:1052700080E28A95F1F7589A0895FC012AE02A9570
:10528000F1F728E090E080E031E040E14A95F1F765
:10529000880F489B02C08160932700C0000040E156
:1052A0004A95F1F7215089F720E12A95F1F729B1C4
:1052B00000C0000030E13A95F1F72170922720817B
:1052C000920F90830895EF92FF920F931F93CF93C5
:1052D000DF931F92CDB7DEB719828C017C01E60EF9
:1052E000F11C0E151F0551F00E942F29CE010196C9
:1052F0000E943D29F80181938F01F3CF81E09981CC
:10530000911180E00F90DF91CF911F910F91FF904D
:10531000EF900895509A589A08955098589AE89A9C
:10532000E9E6F0E080818C7F80830895615091E010
:1053300001C0990F6A95EAF720E031E0992361F006
:10534000492F482319F0589A232701C0589840E262
:105350004A95F1F79695F2CF222311F0589A01C0A1
:10536000589880E28A95F1F758980895FF920F9324
:105370001F93CF93DF93EC018C01060F111DC01713
:10538000D10741F0F9900E94372968E08F2D0E94E3
:105390009629F5CFDF91CF911F910F91FF9008953E
:1053A0001F920F920FB60F9211240F931F932F93FA
:1053B0003F934F935F936F937F938F939F93AF939D
:1053C000BF93EF93FF93CF93DF931F92CDB7DEB7D9
:1053D00019820E942F29CE0101960E943D29082F93
:1053E000069506950695902F96959570202F257019
:1053F000920F292F237096959695920F8770891397
:105400005FC0898181115CC0083008F059C080E11B
:105410008A95F1F7589A509A82E08A95F1F700C080
:10542000589888E0089F80011124D801A050BF4FF0
:105430001696ED91FC9117973097A9F0609179013C
:1054400070917A0114962D913C911597260F371F74
:1054500011968D919C911297680F791F13964C911C
:1054600013978C910995F801E050FF4F63816623F3
:1054700051F08091790190917A0124813581820FD8
:10548000931F0E94B6290E94372980E18A95F1F77F
:1054900058985098589A80E18A95F1F7F801E050B1
:1054A000FF4F6081662351F08091790190917A01DC
:1054B00021813281820F931F0E9463290E942F292C
:1054C0000F90DF91CF91FF91EF91BF91AF919F919D
:1054D0008F917F916F915F914F913F912F911F918C
:1054E0000F910F900FBE0F901F9018950F931F9361
:1054F000CF93DF93883091050CF06DC0EC01F894E8
:10550000509A589885E08A95F1F700009C2F96955F
:1055100095702C2F2570920F892F837096959695F4
:1055200023E0CC0FDD1F2A95E1F7980F8E01092BA0
:105530000E94372984E08A95F1F700C068E0802F47
:105540000E94962980E18A95F1F75098589A4899D7
:1055500002C000C0FCCF87E090E0489B08C00197E4
:1055600021F4509A589A789436C000C0F6CFFE01C4
:10557000E050FF4F6381662381F080917901909123
:105580007A0124813581820F931F0E946329811142
:1055900004C0509A589A78941FC00E942F2980E224
:1055A0008A95F1F75898509A80E18A95F1F7C050A2
:1055B000DF4F6881662351F08091790190917A01E3
:1055C00029813A81820F931F0E94B6290E943729B0
:1055D000789481E001C080E0DF91CF911F910F911D
:1055E0000895F999FECF92BD81BDF89A992780B5AB
:1055F0000895A6E1B0E044E050E00C942B2BA8E124
:10560000B0E042E050E00C942B2B262FF999FECF0E
:1056100092BD81BDF89A019700B4021639F01FBA05
:1056200020BD0FB6F894FA9AF99A0FBE0895039622
:10563000272F0E94062B0E94052B252F0E94062B48
:10564000242F0C94062B0196272F0E94062B0C94D6
:10565000052BDC01CB01FC01F999FECF06C0F2BDA0
:10566000E1BDF89A319600B40D9241505040B8F720
:105670000895DB018F939F930E94B72BBF91AF9149
:10568000A29F800D911DA39F900DB29F900D11249C
:105690000895AA1BBB1B51E107C0AA1FBB1FA61779
:1056A000B70710F0A61BB70B881F991F5A95A9F7CB
:1056B00080959095BC01CD01089597FB072E16F4B7
:1056C000009407D077FD09D00E94492B07FC05D034
:1056D0003EF4909581959F4F0895709561957F4F09
:1056E0000895A1E21A2EAA1BBB1BFD010DC0AA1F23
:1056F000BB1FEE1FFF1FA217B307E407F50720F03B
:10570000A21BB30BE40BF50B661F771F881F991FB5
:105710001A9469F760957095809590959B01AC01FE
:10572000BD01CF010895EE0FFF1F0590F491E02D0C
:1057300009940E94A12B332312F48A1B9B0B0C9417
:10574000B22BA29FB001B39FC001A39F700D811D1A
:105750001124911DB29F700D811D1124911D08957A
:105760000E94A12BB7FF0895821B930B08950E94FE
:10577000A12BA59F900DB49F900DA49F800D911D0E
:1057800011240895B7FF0C94B72B0E94B72B821BEE
:10579000930B0895FC014150504030F001900616E3
:1057A000D1F73197CF010895882799270895FB01F4
:1057B000DC0104C08D910190801921F441505040CA
:1057C000C8F7881B990B0895FB01DC0102C001900A
:0E57D0000D9241505040D8F70895F894FFCF45
:1057DE0000000001000000000000000C01000000AD
:1057EE00000000010D000000000000010E0000008E
:1057FE00040F000000000000011300000000000074
:10580E000814000000000000F4F1F0373392939575
:10581E009431326734973001F2152816F11524169B
:10582E002016EF15F6F501191A1B1C1D1E1F20213F
:10583E00220102010010001010013332363497306D
:10584E00F1F0F4F5F695679337E50100FF010001DD
:10585E000000FFFF0000010001FF00818283E200D3
:10586E00E900EA00B500B600B700CD008301CC0018
:10587E008A019201940121022302240225022602AA
:10588E0027022A02B300B4006F007000000102026A
:10589E0002020606060909090909090F0F0F0F0F63
:1058AE000F15151518191919191919191919192367
:0258BE002400C4
:00000001FF
